:10000000F01F0010753700007137000071370000D5
:1000100071370000713700007137000000000000E8
:100020000000000000000000000000007137000028
:100030007137000000000000713700002516000035
:10004000F5130000F5130000F5130000F513000090
:10005000F5130000F5130000F5130000F513000080
:10006000F5130000F5130000F5130000F513000070
:10007000F51300006D3700006D3700006D3700008C
:10008000DD160000F51600000D1700002517000012
:100090006D370000ED1700006D3700006D37000070
:1000A0006D3700006D3700006D3700006D370000C0
:1000B0006D3700006D3700006D3700006D370000B0
:1000C00008B500230B60036000F002FE08BD08B510
:1000D0000A20002101F0A2FA08BD000038B5094B42
:1000E0000D1C041C1968012001F048FB012001F0DF
:1000F00025FB291C201C02F0CDFE012001F02EFB67
:1001000038BDC046C404001070B5054E051C0E2451
:10011000013C295D301C01F085FD002CF8D170BD3B
:10012000A439000038B5164801F07CFD154C201CA0
:10013000FFF7EAFF144D4221281C01F073FD201C3B
:100140000E30FFF7E1FF4321281C01F06BFD201C5E
:100150001C30FFF7D9FF0D4801F064FD201C2A3048
:10016000FFF7D2FF281C4E2101F05CFD201C383027
:10017000FFF7CAFF616D064801F054FD38BDC04667
:10018000A7390000CC040010AD390000B4390000DC
:10019000BA39000010B5084B041C1968012001F0A1
:1001A000EDFA012001F0CAFA201C02F049FE0120FC
:1001B00001F0D4FA10BDC046C404001008B50020F8
:1001C000FFF7E8FF08BD000010B5041C00F00CFCB0
:1001D000201C00210322034B00F0FAFC00F00EFC6F
:1001E00010BDC0460800001008B5021C02490348B3
:1001F00001F018FD08BDC046CE390000C639000028
:1002000013B59620000201F02FFB1248FFF7DCFF28
:10021000FFF7D4FF1048FFF7E7FF002401F0C2FB0F
:10022000002803D001F000F8002409E00A2001F0C2
:1002300025FA684601A9FFF743FF009B002B03D175
:10024000064B01349C42E9DDFFF7B8FF044801F09A
:10025000E9FC13BDD3390000E23900006F1700003C
:10026000E83900007047000000B5074B89B01A78E4
:10027000064B68461B78064901F0DFFC6846FFF72D
:10028000A3FF09B000BDC046D0010010100000104F
:10029000F339000013B5FFF7E7FFFFF78FFF0024E6
:1002A000684601A9FFF70CFF009B002B2CD0182BF0
:1002B00021D004DC142B0DD0152B20D104E0342BDD
:1002C00012D0352B1BD107E0134B00241A783E2A9D
:1002D00016D806E0104B08E0104B00241A78062AC6
:1002E0000ED801321A700BE00C4B1C78002C07D092
:1002F000013C1C7003E0FFF761FF282400E00024AC
:1003000000F05EFBFFF7B0FFC820013401F0B6F942
:100310001D2CC5DD13BDC046D0010010100000101B
:1003200073B5124B041C1249186803F0A5FA114961
:100330000090114A114B201C01F07FFC00F0AAFD37
:10034000002812D000F0C2FDFA218900051C03F03C
:1003500093FA061C201C01F0BDFC094B20187343C6
:100360000849EB18321C01F068FC73BDC80400108A
:1003700040420F00013A0000CE3900000E3A000062
:1003800018FCFFFF123A000070B5051C0C1C161C6F
:1003900000F02AFB291C201C0022064B00F018FC50
:1003A000301C01210922044B00F012FC00F026FB56
:1003B00070BDC046080000101400001010B590B0C9
:1003C000041C6846FFF7ACFF69466A46201CFFF72D
:1003D000DBFF10B010BD000073B518200021FFF73F
:1003E0007DFE464E464D00249836012001F0B6F9B8
:1003F000002C01D0002000E00620012101F00EF9C0
:10040000684601A9FFF75CFE009B002B21D1002C60
:10041000F0D13368002B0DD03A4B00941A6811329A
:100420001A6004E002F0B6FC009B01330093009BCD
:10043000102BF7DD344BED18DED518200021FFF727
:100440004DFE2E4B94331C6863425C4100F080FAF1
:10045000CEE7002C06D0182BC7D12C48FFF7C4FEDE
:1004600000F0D4FA009B182B2BD1019B00220192A3
:10047000822B22D004DC322B0ED0732B20D119E03A
:10048000832B0FD0C22B1BD1214B1968013119606E
:10049000032916D11A6014E01E4B01201B68C01AF4
:1004A00000F03AFD0120FFF789FFFFF787FEFFF715
:1004B0000EFE06E0FFF7A4FE03E0FFF7EBFE00E010
:1004C000019300F015FD144B0120196801F056F955
:1004D000012001F033F90098019902F0DBFC074B91
:1004E00094331B68002B03D100F032FA012402E0A0
:1004F00003F0DAF80024024D77E7C046CC04001080
:1005000020BF0200000300100CFEFFFF1D3A000098
:10051000A801001020000010C404001013B501F061
:1005200009FC00F0A1FB00F071FA00200421012277
:1005300000F0A2FE0020021C042100F0EBFE0020CF
:100540000521012200F098FE0020021C052100F088
:10055000E1FE1348002100F001FF0021114800F0E6
:10056000FDFE00F027FC00F06BFE3C24201CFFF792
:1005700025FF013C1E2001F081F8022CF6D101F08C
:1005800021FC02F025FB1E23009310230193064853
:1005900006490022064B02F0D5FBFFF71DFFC046BF
:1005A000984004409C40044029370000C1000000EE
:1005B0000003001000B500E001300378202BFBD0D1
:1005C00000BD00B5031C303BDAB2092A01D8181C63
:1005D00008E020231843031C613B5738052B01D941
:1005E0000120404200BD70B50E1CFFF7E3FF00255F
:1005F000041C06E0FFF7E5FF002805DB2D0105439D
:10060000013420780028F5D13560201C70BD000031
:1006100008B500F05BFC011C014801F003FB08BDBC
:10062000273A000000B5C300181A064BC01807236C
:10063000013BC25C002A03D1002BF9D1012000E06C
:10064000002000BD680500107FB5194801F0EAFAE6
:1006500000250326354219D1281CFFF7E3FF0028A7
:1006600010D0681CFFF7DEFF00280BD0A81CFFF796
:10067000D9FF002806D0E81CFFF7D4FF002801D0DE
:1006800004350FE00B48291C01F0CCFA291C684600
:1006900001F0BCFB6846FFF737FD074801F0C2FADE
:1006A0006C1C251CFF2DD5DDFFF73CFD7FBDC04632
:1006B000CE390000333A0000D261000070B50E1C44
:1006C000FFF778FF0D25041C2078FFF77AFF00283C
:1006D00007DB01347055013DF6D2201CFFF76AFF9D
:1006E00000E0002070BD000030B5464C87B02368A4
:1006F0000868002B06D1444801F094FA02F068FA29
:10070000012357E0012B12D10379202B07D0002BB6
:1007100005D03E49042201F0F0FA002803D1394BFC
:100720001A6801326AE03A4801F07CFA5EE0037828
:10073000412B1BD1374C0230211CFFF7BFFF002893
:1007400054D00378422B51D1211C02300E31FFF7D7
:10075000B5FF00284AD00378432B47D1211C023033
:100760001C31FFF7ABFF002849D13FE04D2B23D1CF
:10077000294D0230291CFFF7A1FF002836D003784D
:100780004E2B33D1291C02300E31FFF797FF002882
:100790002CD00378472B29D1023005A9FFF723FF7E
:1007A000059B002B22DB2A3D6B651C481C4901F090
:1007B00039FA0023236022E005A9FFF714FF03782C
:1007C000041C202B01D0002B10D10025201C01A9D6
:1007D000FFF774FF0599041C691801A801F02AFBB2
:1007E000002C03D00135042DF0D108E002F0F0F91F
:1007F0000A480C4901F016FA024B00221A6007B0B1
:1008000030BDC046D80200103C3A0000CE3900008E
:10081000523A0000CC040010F60400105E3A0000CA
:10082000683A00006B3A000037B54C6824E0201CA1
:10083000FFF7C0FE01A9FFF7D6FE019B041C002BA9
:100840001DD0D8B2FF2B09DD00F0DEF9051C0198A0
:100850000012C0B200F0D8F9019003E000F0D4F922
:10086000002501900198002802D0291CFFF736FCD2
:1008700023785A1E9341E4182378002BD7D137BD33
:1008800008B5064A012113784B40137001D0044982
:1008900000E00449044801F0C5F908BDB90300109F
:1008A000243A0000723A0000763A000070B5051C48
:1008B00001200821021C00F02DFD07240126012043
:1008C0000821002200F026FD2A1C2241324000208F
:1008D000022100F01FFD01200821021C00F01AFD7A
:1008E000013CECD270BD10B50021041C0A1C022092
:1008F00000F010FD201CFFF7D9FF10BDF7B5012354
:1009000000930023019372B66C46061C02AF01CC23
:1009100050235B421843C0B2FFF7E5FF0020FFF70A
:10092000E2FF1020FFF7DFFFE020FFF7DCFF0025EC
:1009300002200021012200F0EDFC705D0135FFF77F
:10094000B5FF842DF4D18436BC42E0D162B6F7BD48
:1009500008B5AC20FFF7C7FFAE20FFF7C4FFA52006
:10096000FFF7C1FF08BD38B50D1C041C012200F0C3
:1009700083FC291C201C012200F0CCFC38BD08B5EA
:10098000AF20FFF7B0FFA420FFF7ADFF08BD08B50B
:10099000AE20FFF7A8FF08BD10B5041CF820FFF734
:1009A000A2FF201CFFF79FFF10BD10B5041C812083
:1009B000FFF799FF3F202040FFF795FF10BD000093
:1009C00008B5074B20201B781843FFF78CFF0A203F
:1009D00000F054FE034B1878FFF7E7FF08BDC04650
:1009E00010000010D001001008B584220248002138
:1009F000520001F04FF908BDBA03001008B50248D3
:100A0000FFF77CFF08BDC046BA03001008B50120FF
:100A10000821FFF7A8FF00200221FFF7A4FF022012
:100A20000021FFF7A0FF02200621FFF79CFF032013
:100A3000011CFFF798FF0320011C002200F06AFC54
:100A400002200621002200F065FC0621012202207E
:100A500000F060FCFFF7C8FFFFF7D0FFA220FFF710
:100A600042FFA020FFF73FFFC020FFF73CFF002020
:100A7000FFF792FF0A2000F001FE4020FFF733FF4E
:100A80002C20FFF730FF322000F0F8FD2E20FFF77A
:100A90002AFF322000F0F2FD2F20FFF724FF0A206A
:100AA00000F0ECFDFFF78CFFAF20FFF71CFFA42048
:100AB000FFF719FF08BD000000B50F290ED88328E5
:100AC0000CD8CB08842253430722C0181140044B92
:100AD00080220A41111C1A5C1143195400BDC04602
:100AE000BA030010F0B55B18DBB216E08425CC0821
:100AF0006C4307270F40802504193D41EFB2A6182B
:100B00009C4605E0064BE5182B7801343B432B70DF
:100B1000B442F7DB01316346C9B29942E6D3F0BD76
:100B2000BA030010F0B589B0059106921C1C5D68EF
:100B3000DB78834202D22478039444E0A378234AEA
:100B4000C01A0023954209D1430018180323451900
:100B5000039309E02A7801330232AD188342F9DBAE
:100B600069782B7803910235EB18002604930196DF
:100B700025E0082F05D1049A954224D02E7800272D
:100B80000135F30706D5029A069B0798D118C9B21A
:100B9000FFF792FF0299761001310291013707E0C9
:100BA000002202920199059A08278B18DBB207935D
:100BB000637802999942DCDB019A01320192019B30
:100BC00003998B42ECDB039809B0F0BD853A000035
:100BD000F0B585B0061C0C1C0292039301F07AF864
:100BE00000250190832708E0705D211C029A039B79
:100BF000FFF798FF013024180135A74202D3019B6B
:100C00009D42F1D305B0F0BD00B50F230209184095
:100C10008000031F00D52833002B0EDB511E03205C
:100C2000884280414042002807D1242B06DC042161
:100C30008A1A0349CB18985C00E0002000BDC0462A
:100C40003242000070B5064E051C0024A05D054B25
:100C5000291CC018013400F081FB0A2CF6D170BDAC
:100C60006E42000000400440F8B51020FFF7EAFF94
:100C7000094C271C143725786678281C311C002263
:100C800000F0FAFA0234281C311C012200F042FB69
:100C9000BC42F0D1F8BDC0465A420000F8B50B4C3A
:100CA000271C143725786678281C311C012200F097
:100CB000E3FA0234281C311C002200F02BFBBC425A
:100CC000F0D10020FFF7BEFFF8BDC0465A42000039
:100CD000F0B589B0002404900591FFF7C5FF02200C
:100CE000072101220694079400F0C6FA022007218A
:100CF000221C00F00FFB201C0B2100F0E1FAA042A7
:100D000002D11823069301240021264D03916A780D
:100D10002F78111C0192381C012200F0ADFA381C0A
:100D20000199002200F0F6FA03231F4E029314E00B
:100D30003078717800F0C4FA002807D103991B4A73
:100D4000A3008A5C183369465A500134029A039B07
:100D5000013A013302920393023EE30F0021012284
:100D6000A2424B41DBB28B4202D0029B8B42DFDAC4
:100D7000381C0199002200F07FFA0199381C0122E9
:100D800000F0C8FA0A4902358D42C0D1201E06D0B3
:100D9000069B049A05991360079B01200B6009B01C
:100DA000F0BDC0465A42000030420000324200000E
:100DB0006E42000008B50120021C0B2100F05CFA15
:100DC00001200B21002200F0A5FA032002210122BC
:100DD00000F052FA03200221002200F09BFA08BD25
:100DE00037B5234B10211A68051C8A431A60214B22
:100DF0008022196892010A431A6001200B21002207
:100E000000F03AFA01200B21002200F083FA1A4B7D
:100E10009F211A68194C8A431A601A6818491A6087
:100E2000184B186802F028FD8023000218432A1C82
:100E300020600221032000F06DFA142000F01EFC57
:100E40002368FF229343236023680F4A13432360E0
:100E50000E4B1A680192019A002AFADA22680C4BAA
:100E600013402360FFF7A6FF01980004800D3EBDEC
:100E700038820440808004409840044000C0014013
:100E800000093D00C8040010800000012CC0014092
:100E9000FFFFFFF810B50C4C2068002813DA002083
:100EA0002060FFF79DFF0A280ADC0120FFF798FF6A
:100EB0000138C023FF385B00984201D8012323602A
:100EC000FFF778FF206810BD1C00001008B5FFF781
:100ED000E1FF011E08D00120FFF782FF011E03D0B1
:100EE000024802F0C9FC011C081C08BD50BB1200DE
:100EF00008B5FFF7CFFF00280AD0FFF7E7FFFA2277
:100F0000031C0021C00FD2009A424841014B1860D7
:100F100008BDC046D401001010B500280DD0254BE7
:100F200080211A688A431A60234A012311681942F2
:100F3000FCD0224B03221A6001E0204B1860204BAA
:100F4000012200211A6019601A6019681142FCD050
:100F50001C4B01221A601C4A80211468490221435B
:100F600011601A1C002804D1124B802419682143F7
:100F70001960164B196888421AD01860002801D0F1
:100F8000134800E01348116802F028FC124C21219C
:100F9000206002F071FC114B18609620000200F0F6
:100FA00063FCFA212068890002F066FC00F04CFB2B
:100FB00010BDC046388204400C800440708004405C
:100FC0007480044078800440808004402000001039
:100FD000006CDC02001BB700C8040010C404001041
:100FE00008B500F03BF9134B00211A68120B1203ED
:100FF0001A60114B1A68120B12031A600F4B1A6811
:10100000120B12031A600E4B1A68120B12031A60AD
:101010000C4B012219600C4B1A6019601A60196898
:101020001142FCD0094B23221A600120FFF774FF04
:1010300008BDC04600800050008001500080025072
:1010400000800350408004404480044008800440F5
:1010500070B50F490F4800F0E5FD0F4800F0E2FDC4
:101060000E4E0F4D00242B196159DA68301C0A4BC3
:10107000143400F0D7FD782CF5D10A4800F0D2FDE9
:1010800000F018FB011C084800F0CCFD70BDC04604
:10109000CE39000078420000CA4200008A420000B7
:1010A0002400001095420000B7420000F0B53C4B10
:1010B0008BB01D68002D3AD03A4B02901B6801207E
:1010C0009B685DE001342378202BFBD0002B3AD0C5
:1010D000B30008336A469C500136FF2D01D135E03C
:1010E00001342378202B01D0002BF9D1202B02D101
:1010F000002323700134012E1BD12A4F2A4B0722D3
:101100003B6001923D1C09E02B680298196800F0D1
:1011100003FE002808D02B6814332B60019B013B91
:101120000193002BF0D132E03B681D7901E0041CF3
:101130002E1C2378002B06D000230722B2425B41ED
:10114000DBB2002BBFD1002E1CD000E00025154CD7
:10115000022E05D10398154900F0DEFD002801D0CC
:10116000AE420AD823681248D96800F05BFD2368B4
:101170001048196900F056FD04E02368F0B29B683E
:1011800002A99847064B1B68002B07D103E0019882
:10119000011CFFF75DFF084800F044FD0BB0F0BDF7
:1011A000D8020010E002001024000010C442000029
:1011B000C6420000633A0000CD42000038B5041C6E
:1011C000154D0A2808D002D808281CD110E00D2897
:1011D00002D07F2817D10BE02B6800221A700F482D
:1011E00000F020FD0E4C201CFFF760FF2C6012E089
:1011F0002A680B4B9A420ED90A48211C00F012FDB6
:101200002B68013B06E00748211C00F00BFD2B6812
:101210001C7001332B6038BDDC020010CA42000094
:10122000D8010010D942000008B503E000F098FB97
:10123000FFF7C4FF00F0B6FB0028F7D108BD00009F
:1012400008B5034A034B04481A6000F0EBFC08BDE4
:10125000D8010010DC020010CD420000044B4021F8
:101260001A680A431A60034B01221A707047C0467D
:1012700080800440E402001070B50E4B061C1B7801
:101280000D1C141C002B01D1FFF7E8FF013E022EBC
:1012900003D8094BB600F35800E0084B1A68012C3C
:1012A00003D1AC4014431C6003E00124AC40A243D2
:1012B0001A6070BDE40200105C4300000080005022
:1012C00038B50F4B051C1B780C1C002B01D1FFF708
:1012D000C5FF0020032D11D8281C012302F06AFA53
:1012E00002040608074A04E0074A02E0074A00E051
:1012F000074A1068A3401840431E984138BDC046B5
:10130000E4020010FC3F0050FC3F0150FC3F025043
:10131000FC3F035070B50E4B061C1B780D1C141CB3
:10132000002B01D1FFF79AFF013E022E03D8094B93
:10133000B600F35800E0084B1A68012C03D1AC400A
:1013400014431C6003E00124AC40A2431A6070BD4A
:10135000E402001068430000FC3F005038B5084B21
:10136000041C1B780D1C002B01D1FFF777FF2368AD
:1013700018229343236023681D43256038BDC0466F
:10138000E40200101F234209184001238340181C67
:10139000014B9200D050704700E100E01F2342094A
:1013A000184001238340181C2032024B9200D05079
:1013B0007047C04600E100E0054B3F221A60054B34
:1013C00001221A60044B40211A688A431A60704750
:1013D00024800440D88004403882044008B5044B7F
:1013E00040211A688A431A60FFF7E6FF08BDC0462D
:1013F0003882044008B5154B1868FFF78DFD0720AB
:10140000FFF7CCFF0820FFF7C9FF0A20FFF7C6FF50
:101410000C20FFF7C3FF0B20FFF7C0FF0920FFF7E9
:10142000BDFF0B4A0023136001210A4A49421160A3
:10143000094A1360094A1360094B01221A60094BDB
:101440001A6801321A60C04608BDC046200000106C
:10145000048204400882044004C000403CC00040B4
:1014600000C00040E802001008B5FFF717FC0A486A
:101470000021FFF773FF09480021FFF76FFF0848BD
:101480000021FFF76BFF07480021FFF767FF0648C1
:101490000021FFF763FF08BD0840044000400440FE
:1014A000AC400440144004401C400440F8B5071C04
:1014B0000C1C72B6FFF7D8FF434B1A68434B1A60F7
:1014C000002F01D0424B00E0424B434A04211360FD
:1014D000424B434D1A680A431A6000232B609C421A
:1014E00018D00720FFF74EFF0820FFF74BFF0A2018
:1014F000FFF748FF0C20FFF745FF0B20FFF742FFE7
:10150000384B394A19680A401A602A68EC235B0193
:1015100013432B60002F4FD0344B354C35490026F8
:101520000E60201C1E60311CFFF718FF301C0921C3
:10153000321CFFF7A1FE301C0921321CFFF7EAFE26
:101540002D4B8022196811431960236807218B43B2
:101550002360236802210B4323607B00DB19990180
:101560005B189B002549DF19254B0F60032119608B
:10157000244B2549186801401960196809200A435D
:101580001A60FFF7FFFE174A802311689B0019437A
:1015900011602A68022113431C4A2B600123136047
:1015A0001B4A11601B4A13491360166013601068D0
:1015B0001842FCD001230B60174B012252421A60E3
:1015C00062B630BFF8BDC046388204403482044061
:1015D000BF180000FF1800003082044010ED00E04A
:1015E00004820440008204407FE2FFFF0440014087
:1015F0006440044004C000408080044018C00040A3
:1016000014C000403CC000400FF0FFFF7880044051
:1016100070800440748004400882044008B5FFF7DD
:1016200045FF08BD00B5064B1A6801321A601B68F9
:10163000013303D1034B1A6801321A6000BDC04662
:10164000F0020010EC02001000B5074B98420AD8D7
:10165000064A00231360064A01381060054A1360E9
:10166000054B07221A6000BDFFFFFF00F0020010CB
:1016700014E000E018E000E010E000E000B50C4AE3
:101680001368002800D10120C1438B4204D809E02F
:1016900011688142FCD301E0591C08181168994275
:1016A000F6D203E01168C91A8142FBD300BDC046DF
:1016B000F002001010B5064BFA211868054B89009E
:1016C0001C6802F08BF8044B5C43201810BDC04628
:1016D000F0020010EC02001037894100034B012298
:1016E0001A60034B1A6801321A60704700C000404C
:1016F000F4020010034B01221A60034B1A680132F6
:101700001A60704700000140F8020010034B0122EC
:101710001A60034B1A6801321A607047004001409A
:10172000FC020010034B01221A60034B1A680132BD
:101730001A607047008001400003001000B50028C7
:1017400003D1044B01221A6003E0012801D1024BAE
:10175000186000BD044001400480014000B500282D
:1017600002D1044B186004E0012802D1024B002290
:101770001A6000BD044001400480014010B50028FB
:101780000FD1124B80221C68920022431A60104B2A
:10179000032218600F4B19600F4B1A608022D2028F
:1017A00011E0012811D1094B80221868D2000243B0
:1017B0001A600A4B00221A60094B03221960094B78
:1017C0001A6080221203084B1A6010BD808004400A
:1017D000FC020010184001401440014000030010BA
:1017E000188001401480014000E100E008B5184B6A
:1017F0001A680E231340062B0DD1164B9E221B6830
:10180000DBB2134204D0144A5360144B1B681EE031
:10181000D9071CD501E0042B05D1104B1868C0B2C4
:1018200000F0AFF813E00C2B06D10B4B8022596867
:1018300052000A435A600AE0022B08D1054B1A688D
:10184000054B910601D5002200E001229A6008BDF7
:101850000880004014800040040300100080004015
:10186000004870470403001070B5294C294B8022B2
:101870009203DA67061C0021201C902200F00AFA6D
:101880000023A360244B07251A68244CAA431A603E
:101890001968012211431960214B1968A943196085
:1018A0001968114319601F4B8021186849010143D1
:1018B00019601D4B1A608322226019681B4B18683F
:1018C00001F08CFF311C000901F088FF1849030A60
:1018D000184A0B60C0B2032310602360164B1D60D2
:1018E000164B186860201C680440602CFBD101E096
:1018F000146800E001201C680442F9D1044B012265
:101900001A700F4B802292031A6005230B6070BD82
:101910000403001004E100E0A44004400C800040F7
:10192000A84004408080044098800440C80400100F
:101930000480004000800040088000401480004087
:1019400000E100E000B5044A202311681942FCD0F0
:10195000024B186000BDC04614800040008000406B
:1019600008B5FFF77DFF827B031C8218D07B9A7B32
:101970000132D2B29A7352B2002A01DA00229A736B
:1019800008BD10B5041CFFF76BFF437BC318DC7365
:10199000437B0133DBB243735BB2002B01DA0023DC
:1019A000437310BD08B5FFF75BFF827B437BD01A02
:1019B000431E984108BD30B5002402E00570013493
:1019C00001301D5D002DF9D1121B131C02E00170C6
:1019D000013B0130002BFADCD043C0170240A018B5
:1019E00030BDF8B5051C0F1C1E1C541E092B01D858
:1019F00000240FE0181C0A2101F0F0FE221C031C39
:101A0000391C281CFFF7EDFF041C2D1805E02F7072
:101A100001340135013A002AF9DC301C0A2101F0B9
:101A200021FF30312970601CF8BDF8B50C1CD917A6
:101A30005F18061C4F40551E092F12D9381C0A2169
:101A4000002B03DA01F0CAFE434202E001F0C6FEB9
:101A5000031C211C2A1C301CFFF7E7FF041C35184F
:101A600013E0002B00DA951E002201E0B45401328D
:101A7000A91A0029FADCEC43E4172C403519002B95
:101A800003DA2D232B7001340135381C0A2101F0B3
:101A9000E9FE30312970601CF8BD73B5069E041C48
:101AA0001D1C3009531E00280AD000901A1C201C4F
:101AB0002B1CFFF7F2FF241805E0217001300134E0
:101AC000013A002AF9DC0F231E40092E01D83036D6
:101AD00004E0002D01D0373600E057362670013083
:101AE00076BDF0B585B0041C0F1C002801D0002184
:101AF000017000256BE0252903D0217001320134EB
:101B000005E05178252904D12170023201340135D4
:101B10005DE0302903D001320292202101E002323F
:101B20000292029E9C4632782D3A50424241B618AB
:101B30000296002205E00A235A438218303AD2B2B4
:101B400001363078031C303B092BF4D90296AE18CD
:101B50006346BE4201D97A1BD2B269280ED006D89C
:101B600063282CD0642809D058283ED119E0752864
:101B70000AD078280FD0732837D11AE01E1D201CF8
:101B80001B68FFF752FF04E01E1D201C1B68FFF7B7
:101B900028FF331C17E01E1D1B68201C0093002328
:101BA00004E01E1D1B68201C00930123FFF775FF36
:101BB000EFE71E1D201C1B68FFF7FDFEE9E71A6812
:101BC000012022700433029A241801322D18117852
:101BD000BD4201D200298ED10023BD4201D2237023
:101BE00005E0013C2370013D01E001256D4205B097
:101BF000281CF0BD10B50C1C131C6421221CFFF71F
:101C000070FF10BD00B5031C9BB00A1C01A8191C75
:101C1000FFF7F0FF632800DDFEE701A800F0A6F85B
:101C20001BB000BD0FB407B504A901C90191FFF7AE
:101C3000E9FF03B008BC04B018470EB403B503AA0B
:101C400002CA0192FFF7D6FF02B008BC03B01847E2
:101C500070B50323041C184205D10D1C041C194245
:101C600001D1934201D3002311E0131C40CD043B6A
:101C700040C4032BFAD8141FA4080134A400032382
:101C800009191A400419EEE7CD5CE554013393427B
:101C9000FAD170BD30B50B040D061D430D430B0288
:101CA0001D430323041C93420DD218420BD1131C75
:101CB000043B20C4032BFBD8141FA4080134A40048
:101CC00003231A400419002301E0E1540133934235
:101CD000FBD130BD00B5002300E00133C25C002A17
:101CE000FBD1181C00BD00B5031C01E0013101331C
:101CF0000A781A70002AF9D100BD30B5031C0024FF
:101D000006E01D5D085D281A05D10134002D02D0C2
:101D10009442F6D1002030BD00B502E00130002B26
:101D200006D00A78037801319342F7D0981A00E080
:101D3000181C00BD08B5FFF753F90B4BFA211868C2
:101D4000890001F099FDFFF77FFCFFF787FAFFF7A5
:101D500045FB96200002FFF787FDFEF757FEFEF7D2
:101D600043FEFFF76DFA08BDC804001010B5041C4F
:101D700002E00134FFF7E6FD20780028F9D110BD1C
:101D800030B5F8238A01DB0013404A05920E134355
:101D9000F8221202114019430A235943CA1083182A
:101DA0001C1CEB345D782478EA336C401B782402E9
:101DB0001C43835C201C58400723194008418005C0
:101DC000800D30BD7047000008B5054B011C9842DE
:101DD00001DD044BC1180448EA38FFF7D1FF08BD04
:101DE000FF17000000F8FFFF7443000008B540181B
:101DF000511A013101F0A2FD08BD08B580188918FB
:101E00009A1A0132FFF724FF08BD000010B5CB007D
:101E1000591A074B0F22C9180023CC5C14400470D8
:101E2000CC5C0133240944700230072BF5D110BD7E
:101E30006805001010B5CB00591A064BC9180023CD
:101E40004278047812012243CA5401330230072B2E
:101E5000F6D110BD6805001030B5B14B87B0D96E12
:101E6000B04D4A1E91416A46D175A96A1A1CC8062E
:101E7000400F0138062807D801F09CFC040C1F1203
:101E800017191C00022409E05A6E16329200D3582A
:101E90001C1C15E05B6E16339B00D45800230FE02A
:101EA0009B6DD46DA3420ADC0AE0022403E00C24FB
:101EB000032305E00D24231C02E00D24EEE70D248E
:101EC0002C6148111F2800D922E16A461732944933
:101ED00001F07AFC2000220028002A002D002F00AB
:101EE000380040004400490051005F0067006F0067
:101EF000770085009300A200B400C300D500D30092
:101F0000E300E600E900F100010105010F01110104
:101F100013011901081C00E08348191C221CFFF75B
:101F200065FFF5E08148F8E70A1C0E3203E07E48C1
:101F300009E00A1C1C32081C111C1A1C231C01F08D
:101F40006DF8E5E07948011C0E391A1C231CFFF7D7
:101F500054FFDDE07448011C0E31EEE70A1C1C3210
:101F6000081C111CF1E70A6E1020002A00D00A207C
:101F70000A1C0E3206E00A6E1020002A00D00A2049
:101F80000A1C1C3200946C46173402900194081C01
:101F900051E001201070086E1022002844D00A225F
:101FA00042E00A6E1020002A00D00A200A1C0E32DD
:101FB0000EE001201070086E1022002855D00A2271
:101FC00053E00A6E1020002A00D00A200A1C1C329E
:101FD00000946C46173402900194081C78E00A6E55
:101FE0001021002A00D00A21504A6846173001907B
:101FF00002910094101C111C1DE00A6E1020002A92
:1020000000D00A20494A00946C46111C17340290F3
:102010001C390194101C0EE0096E01201070102272
:10202000002900D00A2241496846173001900292E7
:102030000094081C002200F0FBFF69E00A6E1020EB
:10204000002A00D00A20394A00946C46111C17342B
:1020500002901C390194101C3AE0096E01201070A6
:102060001022002900D00A2230496846173001901A
:1020700002920094081C00222AE0012010700A6ECF
:102080001021002A00D00A21284A68461730019002
:1020900002910094101C00211AE0009222481CE0DA
:1020A0000092224819E00A6E1020002A00D00A206F
:1020B0000A1C1C3206E00A6E1020002A00D00A20FA
:1020C0000A1C0E3200946C461734029001940020D2
:1020D00000F0D7FF1CE00092081C002104E00D1C5A
:1020E0001C35081C0092291C1A1C231C01F024F822
:1020F0000EE0081C02E00C4800E00C48191C221CF1
:1021000001F033F804E0081C221C191C01F038F817
:102110006B46DA7D024B07B00120DA6630BDC0465F
:10212000CC040010680C0010DA040010E804001061
:1021300010B506490B1C88331A68141C1E34A40001
:102140006050013203210A401A6010BDCC04001017
:10215000054B0320191C88310A68013A02400A60C5
:102160001E329200D0587047CC040010F8B5114DC3
:102170002C1C8C3420680130FFF726FE0E4B012208
:10218000D8629F6AAB6E061C02409A4210D1830748
:1021900003D420680230FFF7CBFFFF239B001E40D3
:1021A000B601BF10044B8C35374301222F60DA6033
:1021B0000220F8BDCC040010680C001030B50C4BA8
:1021C0000C489A6A031C8C331C68D3059B0E91053E
:1021D00000D5403B856E921001210A40AA4204D1ED
:1021E000E3188C300360024BD960012030BDC0463B
:1021F000680C0010CC04001008B5084B5A1CD07FA6
:102200009A1CD27F000112021043DA7F0333DB7F76
:1022100010431B031843FFF78BFF08BDCC040010CD
:1022200038B5FFF795FF064903230F22051C5C18FC
:102230001540013325770011072BF7D138BDC04673
:10224000CC04001008B5FFF783FF034B01228C3349
:102250001860024BDA6008BDCC040010680C001056
:1022600010B5064CA36E002B06D0FFF771FF044B90
:102270008C3401222060DA6010BDC046CC0400100E
:10228000680C001010B5064CA36E002B06D1FFF7AA
:102290005FFF044B8C3401222060DA6010BDC04621
:1022A000CC040010680C001008B5124B1B68002B02
:1022B00000D09847104B5A69002A15DD012A07D132
:1022C000DA69002A04D09A610022DA610A225A618E
:1022D0005B690322191C91430A1E02D0074A01219F
:1022E000D166054A013B5361044B90331A68024B97
:1022F0005A6208BD94030010680C0010CC04001052
:1023000000B5064B5A69002A07DD9A690F21044B74
:102310001140D97712110133DA7700BD680C001033
:10232000CC040010044B597F9A7F090112020A4322
:10233000197F0A435A677047CC04001030B50B1C54
:10234000093B012B0FD8084A00239C18257FC45C49
:10235000A54205D0054B08395A681143596002E07F
:1023600001330E2BF1D130BDCC040010680C0010ED
:1023700008B508290DD0192913D1427808231A422B
:1023800002D00022027002E00F2303700723437083
:1023900005E000231A1CC25401330E2BFBD1FFF7BA
:1023A00049FD08BD1FB50E4B5C6F002802D00F22FF
:1023B000944304435C67FF2C10DC6846211CFFF744
:1023C00025FD6846211CFFF7D3FF054A00236C4614
:1023D000185D9918013308770E2BF8D11FBDC04640
:1023E000CC04001030B5124C0F23656F85B09D43AF
:1023F00005436567082D19D0FF2D17DC6846291C99
:10240000FFF704FD6846291CFFF798FF00231A19FF
:10241000127F69465A5401330E2BF8D16846291CA5
:10242000FFF7A6FF6846291CFFF704FD05B030BD85
:10243000CC0400101FB50F4C616F082918D0FF297C
:1024400016DC6846FFF7E2FC616F6846FFF776FF2F
:1024500000231A19127F69465A5401330E2BF8D102
:10246000616F6846FFF784FF616F6846FFF7E2FC23
:102470001FBDC046CC04001010B50D4C631CD87FA6
:10248000A31CDB7F00011B021843E37F1843E31CFE
:10249000DB7F1B031843FFF797FC0F23021C1A4036
:1024A00022770211134000126377A07710BDC04657
:1024B000CC040010044B5A6E16329200D258121AF5
:1024C00051424A41DA667047CC04001000B5064B11
:1024D0005A6E16329200D1580139D150002901DAD2
:1024E0000D21D15000BDC046CC04001000B5064BF4
:1024F0005A6E16329200D1580131D1500E2901D1B5
:102500000021D15000BDC046CC04001000B5094BDD
:102510005A6E16329200D2580D2A03D11A1C293253
:10252000127805E09A18507F117F0001021C0A43BF
:102530005A6500BDCC04001010B5084B0F245A6E2C
:1025400016329200D1585A6D581814400131047750
:102550000D2902DC5B1812111A7710BDCC04001093
:1025600030B50F4B5A6E596D16329200D2580D2A63
:1025700007D11C1C29342478F020084020435865DA
:1025800007E09818447F057F24012C435C650B11FC
:102590004377034B9A180F231940117730BDC0467B
:1025A000CC04001008B504480022011C1C390D237E
:1025B000FFF723FC08BDC0460405001008B5044819
:1025C0000022011C1C310D23FFF717FC08BDC0467B
:1025D000E804001008B504480022011C1C310D233A
:1025E00000F01CFD08BDC046E804001008B5044812
:1025F0000022011C0E390D23FFF7FFFB08BDC0466A
:10260000F604001008B504480022011C0E310D2309
:10261000FFF7F3FB08BDC046E804001008B5044806
:102620000022011C0E310D2300F0F8FC08BDC0464D
:10263000E80400100C4A0023111C46310B70111CD9
:1026400047310B70111C48310B70111C49310B7054
:10265000111C4A310B70111C4B310B70111C4C3189
:102660004D320B7013707047CC04001000B5074A50
:10267000011C042300208A1804E0D118463109788F
:1026800040000843013BF8D200BDC046CC04001016
:1026900030B5074A00238918012206E0CC18051C32
:1026A00046341540257040100133042BF6D130BD5F
:1026B000CC04001038B50020FFF7D8FF084C051CEB
:1026C0000021207FFFF7E4FF25770420FFF7CEFFEE
:1026D0000421051C607FFFF7DBFF657738BDC0462E
:1026E000CC04001010B50020FFF7C0FF034C20778A
:1026F0000420FFF7BBFF607710BDC046CC0400107C
:1027000010B5054C0021207FFFF7C2FF607F042138
:10271000FFF7BEFF10BDC046CC04001010B5094C39
:10272000231C8C3318680130FFF74EFB064B021C4C
:10273000D8620F231A4022770211134000126377E8
:10274000A07710BDCC040010680C001010B5094C27
:102750000021201C0D22FFF749FB201C0E30002118
:102760000D22FFF743FB201C1C3000210D22FFF738
:102770003DFB10BDCC04001010B50C4B00211A1C01
:10278000187F1C7801312043187701330E29F7D1C7
:10279000936E002B08D0064B1B690D2B04D1137FC1
:1027A000111C29310B70537310BDC046CC040010AE
:1027B000680C001010B50C4B00211A1C1C7F1878F7
:1027C00001312040187701330E29F7D1936E002B89
:1027D00008D0064B1B690D2B04D1137F111C293126
:1027E0000B70537310BDC046CC040010680C001071
:1027F0007FB500230C4A0D251C1C1118097F0130E0
:102800006E469955C60F8542664176420133111CCA
:1028100030400E2BF1D100236C46185DCA180133ED
:1028200010770E2BF8D17FBDCC04001010B5074BEC
:102830005A6E16329200D1585C1801392077D15067
:10284000002901DA0D21D15010BDC046CC04001082
:10285000034A0023111C943198320B6013607047B7
:10286000CC040010034B012194331A684A401A60CB
:102870007047C046CC040010044A002313678C3212
:102880001360034B0122DA607047C046CC0400108D
:10289000680C001008B59A4B0F20996A994A8B1062
:1028A00018408911013852560E2800D9C1E000F0B5
:1028B00081FF08111A2327C02EC0C037C0C0C03BFB
:1028C0003F00002A00DAB4E08F4B9A184032002310
:1028D0009371A9E0002A00DAABE08B4B01209A1833
:1028E00040329071A4E0002A00DAA2E0864B9A18E8
:1028F00040329279DA6697E0081CFFF797FF93E081
:10290000002A00DA95E0101CFFF7D4FD8CE0002AC5
:1029100000DA8EE07C4B596E16318900CA5083E094
:10292000081CFFF75FFD7FE0081CFFF73BFD7BE025
:10293000002A00DA7DE0101CFFF75AFF74E0724BAA
:1029400001209833186073E0FFF7E0FD6CE0FFF7BB
:1029500093FF69E0FFF726FE66E0FFF7EDFD63E019
:10296000694B00225A665FE0FFF728FE5CE0FFF744
:10297000F7FD59E0644B0120586659E0FFF72AFE45
:1029800052E0FFF7CBFE022052E0FFF72FFE4BE0B4
:10299000FFF732FC48E0FFF735FE45E0FFF7D6FED3
:1029A00042E0FFF73DFC3FE0FFF738FE3CE0FFF779
:1029B000A7FC39E0544B00221A6635E0FFF7B2FC61
:1029C00032E0514B0120186632E0FFF741FF2BE067
:1029D000FFF730FD28E0FFF745FF25E0FFF74CFD4E
:1029E00022E0FFF78DFE1FE0FFF73AFC1CE0FFF747
:1029F000C3FE19E0FFF776FE16E0FFF743FC13E095
:102A0000FFF7D8FE10E0FFF715FE0DE0FFF74CFCD6
:102A10000AE0FFF75BFD07E0FFF74CFE04E0FFF77D
:102A200065FD01E0FFF70EFC012001E001204042BE
:102A300008BD982BBED03EDC382B9BD01DDC1C2B58
:102A400000D187E70CDC0C2B00D178E702DC002BEF
:102A5000EAD0EBE7162B00D176E7182BE6D176E724
:102A6000282B00D17CE702DC262BDFD175E72C2B4D
:102A700000D179E7362BD9D179E7662B00D18AE7E7
:102A80000CDC4C2B00D17CE702DC3C2BCED175E773
:102A9000562B00D179E75C2BC8D179E76C2B00D19C
:102AA0007FE702DC682BC1D178E7762B00D17BE78A
:102AB000882BBBD17BE7E62B00D19BE726DCC82B1C
:102AC00000D188E70CDCA82B00D17AE702DC9C2B34
:102AD000ACD173E7B82B00D177E7BC2BA6D177E751
:102AE000D62B00D17DE703DCCC2B00D09EE775E729
:102AF000D82B00D178E7DC2B00D097E777E7C046EA
:102B0000680C001074610000CC040010F32B00D19D
:102B10007CE70EDCEC2B00D172E703DCE82B00D065
:102B200084E76AE7F12B00D16DE7F22B00D07DE757
:102B30007AE7F62B00D16FE703DCF52B00D075E7C1
:102B400067E7F72B00D16AE7F82B00D06EE769E75B
:102B500038B5184C231C8C331868FFF735F9E26E32
:102B6000154BA2660022E266DA6003229862251CF9
:102B700010401C1C022809D090420AD0012802D023
:102B8000FFF788FE07E0FFF7F1FA04E0FFF764F9CA
:102B900001E0FFF713FB002807DDE368002B04D1F9
:102BA0002B1C8C331A6812181A6090352B681B186E
:102BB0002B6038BDCC040010680C0010034B0122C0
:102BC000DA660F229A775A771A777047CC0400108A
:102BD00010B5054C0549201C00F0B0FEFFF7EEFFD4
:102BE0000123636610BDC046CC0400109C070000A2
:102BF00000B5074B00201B680F2B08D1054B1A7836
:102C0000824204D11868044B1840431E984100BD0D
:102C10009C000010CC04001000FFFF0038B5164BDC
:102C20001A1C98321268002A04D0144B1D68012324
:102C30001D4001E094331D68114CA3689D4202D1F0
:102C40006268002A16D0002D02D1002B0AD111E0B3
:102C50000C4B1B68002B02D06168281C984700238E
:102C6000636006E0074B1B68002B02D0281C291C60
:102C70009847A56038BDC046CC040010B4030010CE
:102C8000680C0010AC03001013B5002300930193EF
:102C9000244B1B68002B02D0684601A998472249A3
:102CA000009B0878214A00280CD0002B02D0022378
:102CB000137035E01378013BDBB21370002B2FD17A
:102CC0000B7009E0002B0CD11378002B28D0013BAE
:102CD000DBB21370002B23D1154A1360154A136021
:102CE0001EE014490968581A4442604140001070BF
:102CF00011484469021C002C04D08B4202D10A23E3
:102D000043610DE000290BD10A21516101999361C2
:102D1000D161084A1360064B02221960034B1A70F6
:102D200013BDC0469C030010B8030010A0030010A0
:102D30009C0C0010980C0010680C001008B5FFF7F0
:102D4000A3FF08BD30B50A4D049C28600948016006
:102D500009490A60094A1360094B039A1A60094B32
:102D6000094A1C60094B1C60094B1A6030BDC04603
:102D7000AC0300109C030010A8030010A403001073
:102D8000980300109C0000103D2D0000680C0010FE
:102D90009403001008B5084B084A196812688A1A8B
:102DA0001A6006D5FA2252001A60054B1A680132E1
:102DB0001A60FFF733FF08BDA00000109803001051
:102DC000B4030010F7B50E1C0E21051C019200F093
:102DD000B5FD1A4B03240C279E420FDD09236B73AC
:102DE00001232B7328E0301C0A2100F09BFD301CCE
:102DF00029550A2100F040FD0134061C002E06D0A2
:102E0000E30F0022A7425341DBB29342EBD1019A78
:102E1000A31A033B2B70621B2B1C01E0195D597335
:102E2000013BD1180229F9D10F231C1B002301E01B
:102E3000013C2B55032CFBDCF7BDC046FFC99A3B78
:102E4000F8B5104B01221A700F4B0222041C1A70A5
:102E50000E4E0F4D0FE0196891420FD01B682B608A
:102E6000FFF798FFFFF710FF002C04D0013C002C67
:102E700001D13C7005E033682A68024F3978002997
:102E8000E9D1F8BDB8030010A0030010A40300109E
:102E9000B003001070B5264B264C1A1C94321268F1
:102EA000A061E161002A17D118280BD1C32909D1EB
:102EB000214A12680F2A05D1181C38300E2116221B
:102EC00000F098F8A369182B04D1E369332B01D1E2
:102ED00000F03AF8FFF772FE154D0A2363610123F3
:102EE0002C1C2B678C34FFF733FE002801DAFDF72A
:102EF000B9F92268114B9A4203D1FFF78FFEFDF713
:102F0000E6F80F4B1A680F4B10681968884205D015
:102F100012681A60FFF73EFFFFF7B6FE2E6F002E15
:102F2000E1D1FFF77BFE301CFFF78AFF70BDC04682
:102F3000CC040010680C00109C0000106A0C00000B
:102F4000A4030010B003001070B5254C00202368C6
:102F50001D68FFF775FF23681A689542FCD01E684C
:102F6000FFF72CFE1F4B0A221F4C5A6118229A6150
:102F70001522DA61231C903300221A60FFF71EFE2F
:102F80002D3601232367FF36154C184D0AE0FFF755
:102F9000DFFD23682A681968914203D01B682B6003
:102FA000FFF7F8FE23681B689E42F0D10E4C1820F4
:102FB000231C903300211D68FFF76CFF0C4B281C6D
:102FC000196800F059FC3834011C0422201CFFF75A
:102FD000F9FE044B18229A610022281CDA6170BDA8
:102FE000A4030010680C0010CC040010B003001003
:102FF00098030010F0B501240DE005780B1C254066
:1030000006E0C65CED0077083D43C554351C2540FD
:10301000013BF6D5013A002AEFDCF0BD30B504E003
:10302000845C8D5C85548C5401329A42F8DD30BD4D
:10303000F7B5099D0AAC2678089F2C7894461D1C8C
:10304000002A0DD118E063465B5D4A5DD218131962
:1030500001920024B34201DB9B1B0124435501353F
:10306000BD42F0DD0AE0CA5C12190024B24201DB65
:10307000921B0124C2540133BB42F4DD099B1C7036
:10308000F7BDF7B5099E0AAC2778089D347800286B
:103090002FD000292AD01E1C9446002A0ED1013FB1
:1030A00018E063469B5D8A5DD21A131B00240192CF
:1030B000A34201DADB19012483550136AE42F0DD6B
:1030C00037E0CA5C121B0024561C01D13A1C0124B3
:1030D000C2540133AB42F4DD2BE0D15C49420C1BFE
:1030E000211E01D0E1190124C1540133AB42F4DDAA
:1030F0001FE000291BD0181C002A06D10EE00E5C30
:10310000135C0130F31A1C1BE40FA842F7DD10E03A
:10311000CA5C0133141B013462425441AB42F7DDF7
:1031200007E0D15C013349420C1B611E8C41AB426C
:10313000F7DD099A1470F7BD70B5049D01242C7059
:10314000141C002905D10BE0065D0A5D96420BD1E7
:1031500001349C42F8DD05E0815C002904D1013294
:103160009A42F9DD00232B7070BD00B503E04318CF
:103170005B78435401319142F9DB0023435400BD95
:1031800000B504E08318013B1B788354013A8A425E
:10319000F8DC0023835400BDF0B5114B1A785B783E
:1031A000825C1A4000D040220E4C0F49231C261C82
:1031B00004C32C3600221A6001240A1C123117782D
:1031C0005578C75D3D4202D01F6827431F60023219
:1031D00064008A42F3D10433B342EBD10020F0BD46
:1031E00099010010300E0010E500001030B51223D8
:1031F0004B43334A0131D3188A0051181A785C784E
:10320000825C144204D02F4A5F2452189470547088
:103210009A78DC78825C144204D02A4A7C245218C2
:10322000533214701A795C79825C144204D0254AB6
:103230007C245218A33214709A79DC79825C14428F
:1032400007D0204C5F226418251CA235A1342A70B7
:1032500022701A7A5C7A825C144204D0194A7C2467
:103260005218A03214709A7ADC7A825C144204D02C
:10327000144A7C245218503214701A7B5C7B825C96
:10328000144207D00F4C5F226418251C523551346C
:103290002A7022709A7BDC7B825C144204D0094A3B
:1032A0002E245218A43214701A7C5B7C825C134268
:1032B00004D0044B5918F43127230B70002030BD83
:1032C000E5000010A00C0010F8B52D4C071C0025DF
:1032D000201C20214F22FEF7DDFC002D04D0221CF3
:1032E0007C23393223701370231C4F3300210135A6
:1032F00019705034052DEBD1214B2D22181C38307C
:103300000270181C37300270A1209A705A70400069
:103310005F221A541B481A54A320400019541A491A
:1033200008784978385C014204D0191C5331523373
:103330000A701A700024211C381C0134FFF756FF54
:103340000A2CF8D1114D124E00242B786A78FB5CC0
:103350001A4201D0315905E03059FEF7BBFC0D4946
:10336000091A0A310C48043400F0F2FA0235242C10
:10337000EBD10A49084800F0EBFA0520F8BDC04639
:10338000A00C00104101000099010010A4000010E1
:10339000B80000109B010010E00D001084610000D7
:1033A000F0B585B00190FDF71FFB00226B4C6C4F10
:1033B0000092161C754275416A4A009B5D1913689C
:1033C000012B02D0022B02D15EE1654F02E0002BFF
:1033D00000D1CDE0002303AA537023687F210B4066
:1033E0005C2B00D198E02ADC382B00D18EE013DC76
:1033F000072B6AD006DC022B00D193E0062B00D00D
:10340000B6E041E0212B00D184E0232B00D187E0FE
:103410001C2B00D0ACE081E04F2B4ED007DC3F2BC3
:1034200062D0402B62D0392B00D0A1E064E0542B55
:1034300076D05B2B3FD0502B00D099E06AE0732B05
:1034400066D010DC662B3AD005DC5E2B56D0622BA2
:1034500000D08DE062E06F2B3BD0712B52D06D2BF2
:1034600000D085E02DE0792B4AD006DC762B4BD0BE
:10347000772B3DD0742B7BD146E07D2B23D07F2B47
:1034800025D07C2B74D135E031231370022E4BDD17
:10349000231C083B1B681940542908D0032E43D035
:1034A000231C0C3B1A687F231340542B3CD14C2225
:1034B00003AB1A7038E0322335E0332333E0342392
:1034C00031E035232FE036232DE037232BE038235E
:1034D00029E039231370062E26DD231F1B681940AF
:1034E0004723232920D11EE030231CE02D231AE09E
:1034F000412318E0422316E0432314E0442312E062
:10350000452310E046230EE048230CE04C230AE05C
:10351000502308E0522306E04F2304E0552302E045
:103520004E2300E0492313703B1C03A8291C0022F2
:10353000FDF74EFB23681A0605D5E91D0A4800224F
:103540003B1CFDF745FB2368DA0572D5E91D0748EA
:1035500000223B1CFDF73CFB6BE0C046300E001028
:1035600008000010A8010010054300008C61000055
:1035700023680122134206D0A818C0B200210722F6
:103580000223FDF7AFFA23680222134205D0A81DDB
:10359000C0B200210623FDF7A5FA236804210B42DF
:1035A00005D0A81DC0B202220623FDF79BFA2368AE
:1035B00008210B4205D0681CC0B207220223FDF788
:1035C00091FA2368DA0606D5681CC0B204210222EB
:1035D0000623FDF787FA23689A0606D5681CC0B251
:1035E000002102220623FDF77DFA23685A0606D53C
:1035F000681CC0B2042107220223FDF773FA236876
:103600001A0607D5281C09300222C0B20821131C53
:10361000FDF768FA2368DA050BD5EDB2281C0930EE
:10362000C0B20B210A35FDF747FAE8B20A21FDF7CF
:1036300043FA009B01360C33043400930B2E00D068
:10364000B8E6124B1B68002B05D011480021092257
:10365000104BFDF7BDFA104D104E114F0024019A8A
:103660002B78D35C6A781A4206D0A3009859E15DA2
:103670000922084BFDF7ACFA01340235092CEED1D2
:10368000FDF7BCF905B0F0BD064FA3E6D40100106C
:103690008E61000014000010A4000010AC010010A6
:1036A000DC0000100000001038B5FFF7A1FA002878
:1036B00014D006240321201C00F0DEF80321C5B23B
:1036C000201C00F02FF9281CC9B2FDF7F5F9092CD0
:1036D00001D10B24EEE701340E2CEBDDFDF78EF962
:1036E00038BD000070B5041CFFF756FD201CFFF725
:1036F00057FE0A4B1B78002B0ED0201CFFF7E4FD71
:10370000074CC8235B00074EE518211C301C5034C1
:10371000FEF788FAAC42F8D170BDC046B90300107C
:10372000A00C0010633A000000B589B000280ED04C
:10373000FDF725F901A80921FEF768FB684612305C
:103740000A21FEF763FB01A8FFF7CCFF08E0FDF7B5
:103750001EF9044B1B78002B02D00348FEF762FAD7
:1037600009B000BDB90300109061000000B5FEE78C
:1037700000B5FEE708B50A4B0A4A0B4903E010788A
:103780000132187001338B42F9D3084B08490022EB
:1037900001E01A7001338B42FBD3FCF7BFFEFEE75A
:1037A00000000010E9610000D0010010D0010010FD
:1037B0005C0E001002B4714649084900095C4900DA
:1037C0008E4402BC7047C04603B4714649084000AD
:1037D0004900095A49008E4403BC7047002934D07F
:1037E0000123002210B488422CD301242407A142D3
:1037F00004D2814202D209011B01F8E7E400A14290
:1038000004D2814202D249005B00F8E7884201D32A
:10381000401A1A434C08A04202D3001B5C08224302
:103820008C08A04202D3001B9C082243CC08A04273
:1038300002D3001BDC082243002803D01B0901D05F
:103840000909E3E7101C10BC7047002801D00020D4
:10385000C04307B4024802A14018029003BDC0460D
:10386000D90000000029F0D003B5FFF7B9FF0EBC66
:103870004243891A1847C046002941D010B4041C9D
:103880004C40A44601230022002900D549420028CB
:1038900000D5404288422CD301242407A14204D2FF
:1038A000814202D209011B01F8E7E400A14204D2DF
:1038B000814202D249005B00F8E7884201D3401AF6
:1038C0001A434C08A04202D3001B5C0822438C0818
:1038D000A04202D3001B9C082243CC08A04202D382
:1038E000001BDC082243002803D01B0901D0090972
:1038F000E3E7101C6446002C00D5404210BC704722
:10390000002806D003DB0020C043400801E08020EF
:10391000000607B4024802A14018029003BDC04649
:10392000190000000029EBD003B5FFF7A7FF0EBC7C
:103930004243891A1847C0467047C04600B500295F
:1039400005D000230139037001300029FAD100BDF0
:10395000F8B5041CA30719D1231C04CB0F4D104E3E
:1039600050199043021C201C32420FD1181C0B4FDF
:1039700004CBD5199543354208D1181C074F04CB09
:10398000D51995433542F1D000E001300378002B82
:10399000FBD1FEF7A8F9201CF8BDC046FFFEFEFED5
:1039A000808080802578000D0A413A200020202563
:1039B000633A20000D0A4D3A20002020473A202586
:1039C0003032780D0A0025732025730D0A00444D0E
:1039D00031360053455249414C20434F4E534F4CD2
:1039E00045007265616479000D0A4279652E2E2EBC
:1039F0000D0A004C43443A25303269202D202569B8
:103A0000002573202573202025694D485A00563122
:103A10003300202025692E253033695600747572D5
:103A20006E6564206F6E004241543A2025696D56E0
:103A30000D0A000D0A253032782020005761697484
:103A4000696E6720666F7220646174612E2E2E0D80
:103A50000A00426164206D6F64656C0D0A00526556
:103A600061642025730D0A004F4B004641494C45C7
:103A700044006F6666004C434420646562756720AD
:103A800025730D0A00000000005C000C000C7C286F
:103A90007C7C447C241048285408000C00384400E6
:103AA000443800201008103810804000101010001A
:103AB0004000201008384438007C006454484454C6
:103AC000281C107C4C542438542004740C2854288E
:103AD00008543800500080500010284428282844FA
:103AE0002810045408384C5C7814787C54283844E6
:103AF000447C44387C54447C14043844347C107C2A
:103B0000007C0020403C7C106C7C40407C087C7C2D
:103B1000047C7C447C7C14083844787C14684854C9
:103B200024047C047C407C3C403C7C207C6C106CFD
:103B30001C601C64544C7C4400081020447C000829
:103B40000408808080040800784478000708040096
:103B5000000000BF01BF01090500000700070007C2
:103B60000007130A00002000E400FC003F00E7000B
:103B7000FC003F002700040F0800000C011E01FF9D
:103B800003FF032201E201C2190D00000E001F0015
:103B900011019101FF007E00FC00FE0113011101E3
:103BA000F001E0140A0000EE00FF0111011101BF55
:103BB00001EE00E00130011001050300000F000FCD
:103BC0000A050000F800FE03070701040B060000C9
:103BD000000001040707FE03F80F08000000000AB8
:103BE000000E001F001F000E000A11090000100047
:103BF00010001000FE00FE0010001000100804006D
:103C0000000004800780030D070000100010001062
:103C10000010001000100804000000008001800166
:103C20000D07000C000FC003F0003C000F00030F55
:103C3000080000FE00FF01010101010101FF01FE7A
:103C400010080000000002010201FF01FF01000155
:103C50000001100800008601C70161012101310146
:103C60001F010E010F0800008200830111011101E4
:103C70001101FF01EE11090000300038002C002670
:103C800000FF01FF012000200F08000080009F01BD
:103C90001F0111011101F101E10F080000FC00FEFC
:103CA000010B0109010901F901F00F0800000100F1
:103CB0000100C101F1013D000F00030F080000EEFB
:103CC00000FF01110111011101FF01EE0F080000B9
:103CD0001E003F0121012101A101FF007E08040017
:103CE0000000008C018C010804000000048C078C8B
:103CF0000312090000200070005000D80088008CDA
:103D0000010401040111090000480048004800486E
:103D1000004800480048004811090000040104015F
:103D20008C018800D80050007000200D07000002B0
:103D3000000300B101B9010F0006190D0000F800E1
:103D4000FC010603FB06FD0505050505FD05FF0550
:103D50000601FC01F8120900008001F0017C004F0F
:103D6000004F007C00F00180010F080000FF01FF00
:103D700001110111011F01FE01E0110900007C0089
:103D8000FE0083010101010101018301821109008B
:103D900000FF01FF010101010101018301FE007C1F
:103DA00010080000FF01FF011101110111011101B3
:103DB00011010F080000FF01FF01110011001100A7
:103DC000110001120900007C00FE008301010121A5
:103DD000012101E301E20112090000FF01FF0110CE
:103DE00000100010001000FF01FF010A0500000193
:103DF00001FF01FF0101010B0600010001010101AA
:103E000001FF01FF10080000FF01FF0138006C00F6
:103E1000C6008301010110080000FF01FF0100013D
:103E20000001000100010001160B0000FF01FF016D
:103E30000F003C00F000F0003C000F00FF01FF010C
:103E400012090000FF01FF010F001C007000E001DB
:103E5000FF01FF01130A00007C00FE008301010145
:103E6000010101018301FE007C0F080000FF01FF3A
:103E7000012100210021003F001E140A00007C00E7
:103E8000FE0083010101010101038307FE047C049C
:103E900012090000FF01FF01210021007100DF0075
:103EA0008E010001110900008E009F011101110116
:103EB00011011101F301E2110900000100010001EB
:103EC00000FF01FF010100010001110900007F0056
:103ED000FF008001000100018001FF007F11090047
:103EE0000007001F007800E001E00178001F0007D4
:103EF000190D00000F007F00F001E0017C001F00A1
:103F00001F007C00E001F0017F000F120900008318
:103F100001C7016C00380038006C00C70183011133
:103F2000090000010007001E00F801F8011E00074B
:103F30000001120900008101C10161013101190173
:103F40000D01070103010004040200007F010905BF
:103F50000000070000000000070B064400FF0144BA
:103F6000004400FF01440B0600008C001201FF0317
:103F70002201C40D0782004500250092004801443B
:103F800001820C060000E60019012601C000200194
:103F9000070400000000010002080400000000FE09
:103FA0000101020804000000000102FE010B0600EE
:103FB000008800500020005000880B060000200000
:103FC0002000F80020002006030000000400020B7F
:103FD0000600002000200020002000200603000032
:103FE0000000000109050000800160001800060BB8
:103FF000060000FE00010101010101FE08040000AD
:1040000002000200FF010C060000820141012101B3
:1040100011010E010B0600008200010111011101C6
:10402000EE0B060000600058004600FF01400B0642
:1040300000009F00090109010901F10B060000FEC3
:1040400000110111011101E20B0600000100C10184
:1040500031000D00030B060000EE001101110111EB
:1040600001EE0B0600008E00110111011101FE0886
:1040700004000000008C018C010804000000000016
:104080000208010A05000020005000880004010B0E
:10409000060000500050005000500050090500007C
:1040A000040188005000200B06000002000100619E
:1040B0000111000E0D077800860132014902390214
:1040C00042027C0E07800170004C0043004C0070DF
:1040D0000080010B060000FF01110111011101EE2A
:1040E0000B06FE000101010101010101820B06FF27
:1040F0000101010101010182007C0C060000FF01A9
:1041000011011101110101010B060000FF01110055
:1041100011001100010C06FE0001010101110191C5
:1041200000F2010C06FF011000100010001000FF4B
:10413000010804000000000000FF010704C00000A7
:10414000010001FF0E070000FF01180024004200DB
:10415000810000010C060000FF01000100010001C8
:1041600000010E07FF010C003000C00030000C0001
:10417000FF010C06FF01060018002000C000FF012F
:104180000B06FE000101010101010101FE0B06FF0A
:104190000111001100110011000E0C06FE000101BA
:1041A000010141018101FE020C06FF011100110015
:1041B00011002900C6010B0600008E00110111013B
:1041C0001101E20B06000001000100FF01010001E6
:1041D0000B06FF000001000100010001FF0D0703B5
:1041E000001C006000800160001C00030D071F0020
:1041F000600080017C00800160001F0E0783014485
:1042000000280010002800440083010D070300046B
:10421000000800F00108000400030E0781014101BD
:104220002101110109010501030100070008000A2D
:104230000100181110133831303378717073C8C110
:10424000C0C38881808384848782C5C4C7C27574D3
:10425000777235343732151417120207020802013B
:1042600000030109030402040205030500062024DB
:10427000282C383C4044484C4669726D7761726521
:104280002025735F5631330D0A00252D3130732000
:1042900025732573000D0A5479706520273C636FE0
:1042A0006D6D616E643E203F2720666F72207061E5
:1042B00072616D730D0A00557074696D6520257506
:1042C000730D0A003F0025730D0A0D0A00564F5961
:1042D00041474552203E3E200025630048656C70F2
:1042E000004E6F20706172616D73004B65792070B4
:1042F00072657373003C6B6579313E203C6B657968
:10430000323E202E2E2E0044756D70206D656D6F2F
:104310007279006C004C6F6164206D656D6F72790D
:10432000007400546F67676C6520646973706C611A
:1043300079206F757470757420746F20636F6E735D
:104340006F6C65006200526561642062617474651F
:10435000727920766F6C746167650000008001508F
:104360000080025000800350FC3F0150FC3F02508F
:10437000FC3F0350EAB8206AC576500B30E6CC7F8C
:10438000148A7D237D01273779B7D4EFB142483FA6
:1043900096B7CE135D6E6C8869A5720ED2BC012AE9
:1043A000DA45424A528AE39874CA78ED91010813BB
:1043B00029F3901907195099FBD0FB7FCBCB1396AB
:1043C000BCCF860C2D0088656C0771BEBB244F687E
:1043D0005E65CA90F24BEE6F402A7E98747FDBDEFA
:1043E000976A55AD0E230EAF86CE0E1CE3E0136C1C
:1043F000A815F97CFE66F114A16DB53D61EB5DEE8B
:104400007CD9EC211B834070E006FA4D6E5E97EB81
:1044100056A1482F14F3EE1DAD88495E6076201F2B
:10442000B50C0F12CEC7E6D6A83EAFFD343FBAE8B2
:104430006ECD3F441B6543B0863C43009EC9A3B389
:10444000AB6E85AB80470A281CEB9A3813B24A85BD
:1044500087D162031D2E468EC354EF07EDD0B9936A
:104460008C6F505D68893DE6D895B0333373321850
:1044700052357A7B860C56491F7D343D501F2F558F
:10448000525FC1F64102F31C70E6DA3F86981F08BE
:104490004BCAEC91C7C43F4D8A93F30F28FB090A1E
:1044A00071013ED2858C08D5A11FC6B6370F73CCDB
:1044B0003385D03E9F3CF0146C074F944591A6A7DE
:1044C0006F176C5D687464F87B4495D45382CEC8D2
:1044D00004BBC8C23F54D290BB5E9123ACB50279F5
:1044E0002E058FAC37C61D400BD1945D8E266C0D0A
:1044F00058F03E37F504F51F1694ECB9A9A5895379
:1045000005AE299BB6AA2796DBD6A43E821345B7F3
:10451000FA56A9EAE37D3C4BC019456B51FC98EA79
:104520005EA4604C654883A75151A530407FDD856E
:10453000A27B84622AC3FDD2CD851BD9DBB0262B9A
:1045400028BE495528136D4F6897769EBA8371C16E
:1045500086C4FA2281397297B01622387A6CD087D5
:10456000734B2A1AC27750EBF44E3DD557A881E61B
:10457000F9389889FA738B84BE8F509550542BDB91
:10458000355510F15D144E415BAE4A775CB583AF93
:10459000D0A84E97ECF5D588F24589F53920C5DCD1
:1045A0008BF9708343E40599A3F276C7605C43F806
:1045B0002500CC22DC84735628BBCC16D96ACCB338
:1045C00057C65B2DB264A9E5B9B8392F43745A8434
:1045D000AD1412E011C025E4450DE49005B1E8ECFE
:1045E000159C998183A533671945FF07CB854EE656
:1045F000E0A1642505BFD9D559199F7171A6D30CC7
:104600006A6F0505362ED3C184A851916F0209E760
:10461000863F9D438E330CEFBF039F0484CE64839B
:1046200011F66F9BE0D3320BC4A513BAC4D5332166
:10463000032BE4084CE30382C7D695681F3CDF597F
:10464000AD77640A2EB8762CF0EA790AA743D21A1D
:10465000702BB91DA440FABDD1A71AB3632F629A7B
:104660008B13FF9E71D40484A8943D2BC3216ED775
:10467000F2149A2A4A807055B3562220D45EDB5633
:104680000DD9929559B7F9BEED24F1409B09DE2C66
:10469000FE791D7A18AB6F4F43F41D315B7B1AB561
:1046A0001240ADA78B15D9AD9643617AA0C5C10C58
:1046B000078FBEA839AEEAC52B4F81050A840FC209
:1046C000CBCFB3CEDC67DD40208CACEAD761924D16
:1046D00028571D0E3FB2D1C14F015ACD81E7FD735E
:1046E000E296E06A9B9227619F3DEB07935C7D33E6
:1046F000B217CDCA6001F58A7309E48BB086CE8209
:1047000002176B139C87AD8C24862BE6B97F83D070
:104710008C5D215092413C6E4120054BC7CA63F02D
:104720000215CCE893707FFAD7F1574E000442D8B7
:10473000CDD70016FD13636ACA02B0472F44C2D911
:1047400095AB62C5EF9CE0A7FEDAB98BD6AC9D1A9B
:104750009D1987703EACD0413C5CFA47931CA4384D
:104760008847E0D6AADB322CDD644F5DF0F29DDD98
:10477000E1DA7D46FC0E1B967D2B44B9D9D5332357
:10478000AA0CFEA780683B4D1AAE7A0120FE6D4E42
:10479000B97B592568BA8122D74347E744A49FA132
:1047A0004F78FA5781099624C3CDF5F256158788BC
:1047B000B41725C50477D6C9936B49B7A6CD902900
:1047C000DDF0C9005CA303BE7C7518DB8008E077D0
:1047D000FDC12326E9E727497D374121DA9FE3D848
:1047E000935CB56FD5802DFFC1C3013D600C2CA734
:1047F0007B9B28F626EEC79AB1318800D459A804CD
:104800005B7D4AB0CBBDE552AB982A91AC8FB19895
:104810001F75D77686AC58C4CADDDEBB6030FA118E
:10482000DB5B7639B0C72057C2DD57BEAF84F3EFEC
:104830008FB14DEA84E447ED8D837F9D3E7C05A8D2
:10484000CDC65A4D8B4FFC1C24F69D470485BCF801
:104850001874FC28CA48863094EBE774C524626754
:10486000B5A6F7F47557B9409BF2D0B591E98532FA
:10487000839A18C1724E5CFF3B0A3BB0593015EB6E
:10488000EAF411131784DDDF497844ABF2FC41AD43
:104890009D509F578A7E8FD93CAF9678518A79F088
:1048A000BD0B46D4F13ABA76520D6E28D066424B13
:1048B0003FA91E3FCB65614E21054759CAB4E2BBF3
:1048C0009FCEFC1A2774BC69BF5C11937C52972C55
:1048D00042E966855CD7E45D3AD83BBBEF1FE5E172
:1048E0006D10406AF8073C392BCB625FA2762AD95B
:1048F0008F0B1A181166B74FAA82F79B5718980F9B
:1049000080A74AC3D814907D72E803221B1FDC17CE
:10491000183FF6521D739C83CEEB0A02DBB398FF5F
:10492000293BFD470DF5B505D270A476C86113E8A3
:10493000693526EEE34448E504CB190D9800BAC862
:104940003D83A685779E19BFE464877E7A99A5A0EA
:104950003546214913B7E9EDBB8DAD362778597D32
:10496000E40CB8F3D5045A232EAFDB34BD4A751DD1
:10497000BFC9FA95036865AD97C422809751131398
:10498000A895F081E779508A9916A37192C6BBB9B0
:10499000D02C9F8DD1C20C05045B8E87EBDECF9DA2
:1049A0004E1E31D76FB73A5272FBE5761E50A72ED6
:1049B000D48811675D665FD3A842063B5120C0C40E
:1049C000850BA4DA0B7B660CF31260035792F73F5A
:1049D00043067CCF715E45CEDBFC953D9FDF12ED3B
:1049E0001CFFBCEB7D8021B615277884AA2383D4D5
:1049F000484EF069281E6893C761F65C13521A2F5F
:104A0000A4774CF0473BBE45ADCAE34B3D724EE444
:104A1000D5D3D66423D9C2FDDC441875798858866D
:104A2000C5CCD0FB090E8E3CDBF702DD4FFBED5A07
:104A300073E4C5E43934912207E182609B4B25B1D0
:104A400015B3EB996AD8AFBB423118CEBC55C6D46A
:104A5000E2343C5A9D352D941D159FF66FCC553B85
:104A6000047B2B032940A23FC960AC33E09E7370E6
:104A7000CD50B6CEB676DEDAA858C07317E6F91A6E
:104A8000A2B9A26834ACBD1E269C480D51B017F9DE
:104A90009472F9789FA29D9FD62BD6CD1159C76AE3
:104AA000C55429B04D1E7225F3AAB5C408832CCE77
:104AB000021A4006A600620D2D7CECA5C689595E3F
:104AC000A3CB0A7C8AF19D95226E07D55CA97B84D5
:104AD0004AEA44C67638DAF9258FF1C630873318AA
:104AE00088744FEB8C8885799E397C6EA03EB72404
:104AF000F2D581DFC7CB31A187E80B0CCD4113F490
:104B0000A22BA3F32B75D479BEC5CA26D998DD6133
:104B10002C2DD7E71F951587A0BA799BA99BC1A318
:104B20003C95E9BFE99A7513C8B5136B8A9E1C2A98
:104B300077E8C22E970DDF3503E69829BDC1DEE583
:104B4000C67EDDF1D13227CDD1F4C48FEF2E2FA454
:104B50006013FC349EFD456F15E9A2CC3BAE04B654
:104B6000E766A048817B124ED81B9CC7726A32EF61
:104B7000D643BF174806694C16C7739C411A95A9BE
:104B800061AD10807955A89B7E147FEDEBA7D30D06
:104B90004AE06BB895F668B58BCA115AE15FF289A5
:104BA00092CF22FB53A57B214F2D92759F6090F5EC
:104BB000B76D917D44594F49186B40D59AEB9F24AE
:104BC0006C2FBBD0D5019EBF529230ACF628FF4F60
:104BD0002BF950883BD039191D0AC8EC01E21B5B48
:104BE00042BF98C73798FCD4537881D438AA04EDD3
:104BF0009B745D0928206410C22143F925014534C6
:104C0000888E71AA3B9C3515314738C2297EEC1835
:104C10001E4DD93F93B1605D17F9734602C08C0BEE
:104C20006E7AAF6C8F1605A3409BD5169CE14BCED8
:104C30002DB05227C28E8F0C41A5505C4D6D0ADFFE
:104C4000B42D1DA45BCBD2A8621FE840831B417228
:104C5000F446D40BDAC4A53293E9F10E10CA505DC4
:104C6000DF96ACACA395ABBD6AA4538BA9B3061376
:104C700084BBBABF04AF53C00D097082AC7C9FC621
:104C8000376566CE21C38CE972AA0A36B8A238FD10
:104C9000BBC44A2ADE75B22C465C150E546BA5794E
:104CA00029B4847800D4BED326A76F5C0B51D0C042
:104CB000F5E0BFFC7551789B9FC50359D38705D696
:104CC00044B52DB0B302818CB905244DAE46746E47
:104CD000445A524A99084DB26E69363BC8506EF537
:104CE000501217D9BACE170559442C6D797AE2AA19
:104CF0000B1E3057B3C3ED966CF71410D93782866C
:104D000088B000F654448C07E28E8FF2170EC91B50
:104D10003DA75C94992A0704D4E0F6AAD6376CD450
:104D2000B752EFA6B04FC3A52E9B37D294FDF87BA8
:104D300012F962A30DD93D0D37FB3C3F291D01023D
:104D4000140B95697E0DE4720551E18BACF8A03F20
:104D5000B7B59A249015719206354B5BD93819A9CD
:104D6000DFA28D08746C2C431EB82909ECF3FD9565
:104D7000B468B31AEB5253A6DF41CA9A77C4E6ADC2
:104D800074D443023566B3B5EB08E967823522A8CF
:104D9000BFC05644D95DDA0813B2BFE0F2F56534FE
:104DA000E93827A699BB75FFAC75D3FE99F0F0CC16
:104DB0003915339BD59D4783783D0A16D210D744C9
:104DC00099F3AA883A3BC8F7AE8589349522973083
:104DD000A4840918AF5F465D519B9806674B4B262C
:104DE000E9B90405D0C97B1B968C8FA61872924432
:104DF0008EED11267004BF4379DE39193EA4A53F1C
:104E0000BBBD16E3A1193E02A5D00D6A06A0B6A14E
:104E1000D164DA47C2515F0CF3377D78EE580F0149
:104E20003B1CD4B36FBFBAA5FF37DD0AB1BF202C3E
:104E30003E586B21ED9A337E90BEEE21D7C5900F80
:104E4000D04E7506F5727F40732578EE9E8E740FF6
:104E50009AFB74286B24043669CC887053ADC5F96D
:104E6000F45E5747E61E5C525BBE448ACD2D831B21
:104E70008147CB1B35676F3211DC7FC7795F2128F3
:104E8000D357EA1BA47E89D404D1E33B3FEA0D68E3
:104E9000AF1C871A51E533C890EE4F2EDF8BA84424
:104EA000B10217BC210EE6A556F57914BCAD2585D7
:104EB0004A372A3E981705C69090A28D8CE3846FDE
:104EC000D86E16DFABC856BF057E32DD67593FE8A6
:104ED00021818A204F27636AF2720AFE5CF3FF0584
:104EE0001E0F8A68705FE6C5829DACD411AFE00EDC
:104EF00002A633ED772C656066A615040AC7830603
:104F000058503B307548D2DA804D304C6BAAE3B034
:104F10007BA5BBB3408A786BFC42FE5960315BE3F2
:104F20003C6DDE066CB28418CAE2DE526DB67516B0
:104F3000E5DDCAE77DFEF4FE9F82B1F714B8136A7F
:104F40004855A94E935F9719403AF846053CCA1751
:104F50003DC2DA6F5ABEE3B7D31EF3834930BE2495
:104F6000690535BC4DE55BEB7159BE3A8292955FA0
:104F700093BBD8A10035C7F2D18DA5624C820AC17E
:104F800022E6284D71FBD7FA47C2AA03C3FD2408C5
:104F9000FF6285D91F1ADD6DE183BB556F3A895BCE
:104FA000A10E54801CBC8DF0677B982A3E2515B954
:104FB000D2A5417B6CEDA6892FAB93808D0CBFD120
:104FC00030097E3102F4DF16092FAE1EF3F5515F72
:104FD0005E23F170E45F4B944EA1C9E6533D0D7220
:104FE0003E0026A7ED34E336C18C61486BD05153A7
:104FF000C28BBB7CE0767FE0E4913AE69F5D13C90B
:105000004C5DA85EEED164FEE810F47471A759946B
:105010009E13D95ADCBC68AE1566E3A7D243329E14
:105020007518E4863AF71BF7139C422E7C8E96493E
:10503000FCED51A8DB07ED7A621931FA9B2D182F90
:1050400056F5926BAFE12EC0BC3C29C7B995FBA4C5
:1050500078F7B6175E5EADBA6B6696DA4BBDB0C533
:10506000806281BDAE5084E4F22728449BFD31D399
:10507000DEE6C5C840A7C744C00C892AE5894BD0E5
:10508000658C6182ED5B206581347C28CEAD0FF0AC
:105090008D60457E3A92AC830C9193F7E15007AD59
:1050A000C9928BDB11738F099451F30679CDF2DD30
:1050B000C50507822E059D692EDC47B20463BDE35A
:1050C0005A04246CC0C139B5E4F3C5F9A225EE2316
:1050D000DF5BF5A57F557D55D015FADBBBFC4F98FE
:1050E000F1AEE0A2DCD4ADDFAC71D9EEA8B462467B
:1050F00057F42FBEC417A1C617A0088B6C17524CCB
:105100006561AD5F621AAD41389372E0C8B6F6F4DE
:105110009CE16C3EFA068F4099F765F531689B4F2C
:10512000F1DD74161BE07B9D5A857FC713B0A886FE
:1051300069967FCC4A43D049F3B85317F08F657610
:105140006D02B34E6BBF75856CB740A387A18A799A
:105150001EB76E552CBACC9B2D06CD858B5423895A
:105160004327F9AC31821FDB26DC13F59639CA5D83
:105170000A0701B56F864A393EFE9594A42E5EF962
:10518000BF028DCF72F98151D407915E3BDB4D9602
:1051900033CA59C9806A72EEE22C0D0E90541C7409
:1051A0004E7FCC9D4F3C7B3B04609B034C5FB873B0
:1051B000A0395E517DD1B10AD11F084FCDA501198B
:1051C00001E084386635D2BC8EDA8B4E20B5CF1C18
:1051D0009DBE589DD1DE66D5F64CE285ABD3D42674
:1051E00061D700066839AD4A997BBC458944923F36
:1051F000B71EDAAA972A8B050638A583D44119E889
:10520000715F2196AD47DF087DC9E2E854D62FE6ED
:10521000C07E1A847129162C0B80D317905DF5D2AD
:10522000CD387196DF60FD1E65DEF0C253667B7E71
:105230007B94280F716BA642C409DEB6C1C9164F14
:105240008AF8CFE34A17F4649A0A4ADFA3184EBFDC
:105250009C9FABBD13544A83F8AB0E1F15802CD80E
:105260003C20D6F88F08C76EDF2814D9680562BDC8
:1052700025BEFA08B212DBD39EAE6ABD5A2AAB999C
:1052800077E7668AF10D791DC02E25D29F8DF51D19
:10529000613037101BFA515DE8BC9158F6723DB190
:1052A0005251E2D239DD1DC424AD8941DCA950330D
:1052B000A40505C7A7AC75F2231BB864DD47C392EC
:1052C000EE85D2B41701081FD2C6BA51E01674A2F7
:1052D000A607A7D38D258977C252875FB25663553B
:1052E000C695A828CEC90D184A4353A7C784B7212D
:1052F000CC0438A3CF4BBAB6D952A3662A4931FDA4
:10530000AE39E288D948C3CD5969CFE0E4CC9D4796
:10531000B9986530D0F2F3F8C6F294842858137E19
:10532000AFDBC64D32D4269C063C8CF1C8ADE337CA
:10533000EE778632CBC4A834A271A5E1B451309483
:10534000E21C211BCC2A2B7B473EC02CFBEA891F89
:105350003B4E5F3D6A3B85E6A2AF6D66DF0BA12247
:10536000CAE22BED412598F15C88452966CEE72DF0
:1053700049B1EB22FE299D8E9E5EA91F78BEFB0ED1
:105380004082F8CDF15211F4A533575ED2E366E2C4
:105390005E871707D10C6FC7F08DEF36A18AA41D69
:1053A000C396CC9FFB5B7A8197F8C3BDC36D111187
:1053B00038FEC238326AE1A5CA906A96A7872C21C6
:1053C000006CD4411B3D5D5196A617CD3BC54F7374
:1053D0004B82E473D8BDEBA5D6366945C66F0F89FD
:1053E0008B14B4E2946326D0044355F5D038289A40
:1053F000BF7D594E8830B7FCA342A1402774B4F456
:10540000B4194201614441168722DEFE847B76DCBA
:10541000E68F68B89485CA2ECF032875812E330E87
:10542000AF273E1FE5E50B49C8B26219481E0E0AB8
:10543000796F779AC87D5CD0D637CE512B285755D7
:105440002D63262C947A50B8167C8C39ECE952F4F2
:105450000131D8A765C9C0EDE4FD0A3350200D190C
:10546000533FD99AD9D390F315BEA0084D6D70CB98
:10547000379B47BABFDAFA687923E7940307A1C9D3
:1054800043D06DEB6F3D8F32461C76521CDFFA1411
:105490003FEB977F39DFE1E8112257EE58AF896083
:1054A00005D04B63EE6DA0343FF1438EFB86A550D3
:1054B000FD5B212A54F53AAB01475D62E24BE17D89
:1054C0006FF6FDDA896F905F86A2BB88CFD35E53FB
:1054D0008504EEA85F22CB4BC5584B6E4DDBBBF766
:1054E000B53820C55B5C04C5750C5AEB7245F049B4
:1054F0004AF72CD1D872E46B3A3AE9BEEAE018C612
:105500006F300B4458192251437C6F261901147EC9
:10551000132E6632A0183614923947613BC4B8B0D6
:10552000ABF792FE61D90500FAD206ABC66C11E06A
:10553000F9D996FECD9BBA6ED29AB2898B9067EB61
:10554000C421516086C8B7652F228AF9509F7E1CFE
:105550003D6DCA40398A9B7F9E3BD79BC3C4CE1406
:10556000F8446572E42D2A5E1A0A6B28CCC6EA1D3F
:10557000DD7E4FFCFC126623780159AEF2ABC3F717
:10558000F9DC9AE983E4092FDD1548334D27DD184E
:10559000C034FAF53AC05B83CAB6728D76BEEF129C
:1055A0009675C774555EE5FC0F4B76ECF265817B12
:1055B00034E0D62EBB3136FFAE5FB348D6101E8A1C
:1055C000CA5C3D3259491562D8B38F002004DE4EC3
:1055D000F595F50A4E53FF95F24C52CFA8C4D63636
:1055E0004073BA2FEA9EE7E144DA5D1E0F47C828F0
:1055F000E206A082D2C786126F0ED36F053687D11E
:10560000F21C9CB8A4F17B6A00730FC86A7B0AF78E
:10561000297EEB1B07DD80D4F363F4D0B9A019BF5A
:10562000A2AE50458A75AB1526A56AD135A8C084AF
:10563000A5642BD80262B2016DCCD13DAE9DE5319F
:1056400011658D18F723C200B64D33536ECAD5ECE1
:105650003D1A167AE38FF7FAB902078833DE6C52E7
:105660002CF7BBE2ECBFCCDB6ED81ED2A26900B92E
:10567000F04D3A853099E941DB1EAE47E8A77861E5
:105680005EEA4A9D770F9FA0689EE5F0C764575D6C
:10569000B5988E838607EDA1BD14E484BEB289EB74
:1056A0002E98B11FB2B3F4EE1205C9103B8B684BB4
:1056B00010B6B74C8D9C7E3C6A01AACB85B7E90E2B
:1056C000EB55339D55B3F814A25E577B3E2EF9A6D9
:1056D000EF7166307946EE590C37A2E4B0118906B5
:1056E000A8126A06A19F3D324BA1321D9B5A293157
:1056F000F93A0CF18CEE2683B336D041130F14F235
:10570000875AFB0EEEBE61399E22B2E2DB5037288B
:1057100020F481995E79402DC18AED9CAA05E24F63
:105720009040E9E75526AA3464BB5204DA706B2F27
:10573000A35BEE1E439C7EEEE8AE55378969D35AD3
:10574000D1643E32469031D8655EFF0D9668CC3EFE
:105750009471B335A0F8A4C7619D232D4DC0B1C489
:1057600047D978E29E5D9847F260125228DB130D0C
:105770004BC14766CB5CA743565D79F720B2C2E7C1
:10578000D01AAE1EFCB5822A9AB3EF0970158A5C56
:105790006A92F4908E1138C984C5C9543B1EE03218
:1057A000642F562D6E3D2D8DEC9D1030F02CE3882E
:1057B00000698352888784297067B34AE63178315B
:1057C000F74E8B0CD884D7360848D8E96B9AEDA4ED
:1057D000D93CD7B2CA9A0230E189DBD5093D0E0D1A
:1057E000B6FFA06660F3BCE50D500261FA13F22328
:1057F000BB41A4F30AAB17EBF538E7A9399B5481F9
:105800001E4D2684D53E2A0C2B58B2AA4B68848F95
:10581000657B67180ABDB857AA5FE159FD10E37FA1
:10582000F07BDBE8F8D88C9197D5E1658C21365B6D
:105830008C8F07D33F7996F4AC5B908981F5023861
:105840008629D854E7DFEDF370C798D58824DA139A
:10585000C2FF3053056E33DD9A82100153BCCF4432
:1058600007864E853F9727B273873ACD21255CAFD7
:10587000632662CDDDC3C1170EE4E43EDD0B0E33BB
:10588000BCF2507EBA9A2BD45BF1CB1436CBE7280E
:10589000A2E59E999B5174B061162A4EF3A28C81A9
:1058A0005C10966C9BD8C93E3983970C0B0FCA9A33
:1058B000CF8389C3E651BA9175CAB3585D3B8C5901
:1058C000CB37F07A58B8A6EE8AFC7A189E2813BE19
:1058D00081B3D926956E29F993C435521C3A8A149E
:1058E0004843B7B97578B823901A15010A055125B0
:1058F0008400E4776526D26CA599FF8AC1892121AD
:10590000DCBE81B7BF219B937857BEDBD674572886
:105910006CDE8A8B615F4DD033A16FDFD2B4779795
:10592000883B7708104890A9BADB94B5264D87715B
:10593000227530815C748A9CB88DE94E8BB70F1844
:10594000EB4453372CA1D0B6F117A7EC0B112CDC8C
:1059500043B3F3DCE2B46C8957578A8173C3537B3A
:10596000430E1FA2249CF5FE1AAB3AE956C60378F3
:10597000B5ABF5150F44F6015C1AA3528DE9699099
:1059800083695B822B5C53C3EB1F673DDAEC06D364
:10599000CFF117BCF1EC478F908621F22AD6FC9FFD
:1059A00059445822AF37FC1479E522F0377256F586
:1059B0004DE0128041DC17333E324E26981A5C8946
:1059C000B786B5A485541AD013736A77499078EBDB
:1059D000A123E05A5007A3C7DA19D2A57FDFEE2131
:1059E000BDF4AD971828785E592C32DF37B695DDB7
:1059F00061DAFB6C6AE0ACF5DA188539A1440F9ED8
:105A00007FD2E0E71E3302626F2FABE553146B8D3C
:105A100023D6ABC2891D2D513F932831659D9D6BC7
:105A2000A9D2FC65EF5B878FCE248510EB15A6A766
:105A3000B60DF598BC4C93D7288FADFE73C8D82807
:105A4000B358F5DDFCF897C7E62A2AEBBE498AFD74
:105A5000B0130D4B594BE84987428EF120FFB567D3
:105A600078561626E253FB23D297BD4D15924F8CE4
:105A70005F9F7B8FCD262A0C36D1105C74BBFFD480
:105A8000683772081A12E5899CC4A7AEFE0BD5953B
:105A9000D83FF9DE146A3B98AC53B71990BF2F3F3B
:105AA0006071336A1787A6EF90B75499B383E57195
:105AB00016B6FDCBA1FF5A7A352B8CE7EC3FDF1EE3
:105AC000B057AEDBD2898FBF89076AA8B55219CF0C
:105AD000A03F6EC6342D2EF694D07ABA9E6826DC8E
:105AE000CF74CCE0D1D6617148A2133D4388618B5D
:105AF000C15F691FB24AEDF778C15169B0F278F120
:105B0000A72A516F183613C1046E80D62BD52FB635
:105B10002AE1C4C40F6333D49D1919C197AF8C64B3
:105B20003DCF2DC5D050F3C213C0D5F112D8988601
:105B30005246BD02C988D9666E15C9E2CCB307BC0E
:105B400000EA56BC3673F0193D9D9FC98F241A9404
:105B500046580A763B95A198F66E5D2BA76DCB3B18
:105B6000380BAFD09F4FAC7AFB6A100ECAEA100513
:105B7000CBDA13D9B140DBA8FA0D1690965ED7F6B2
:105B8000EB588F5559E92BBD8B5F8893902B0C8771
:105B9000971194C72E59923221676B3A8680D9BAF1
:105BA000C3013B5B6963EF914759B453FEF116B8EB
:105BB000AE73B286F3266DD24A215E64E6CF8A21A7
:105BC00061A65C5025A94E38B3DAE9170A23D45CE4
:105BD0004EBE79E1FD5F24A0C58B2968E81ACCF39D
:105BE000ECD06A79325CB96AF4DC46B5125F7900B0
:105BF0002A0E4AE62735CDDC94D42A25D880A695EE
:105C0000813F1EF32F8D4F178EE4958AC05BF4DF22
:105C10005ECE12362F83D33C5D82FDFD7F12DBC248
:105C2000E2C764CDA25BAD9CC304E98DCC926D1339
:105C3000768C14A1EFA48F4A096C31D571778372E9
:105C40002DB36A019D73736B73DC2991CDD96FCE2F
:105C5000A94A6292E57212514365AAE2AB9AB497DF
:105C6000DB981B23C13EDE3E78A005E0FF57375688
:105C7000A8179BEC500A662AA8FB7CD61B8178E209
:105C800010B19AC113DBBE2FD10E0A9A686899DF52
:105C90007488D75F0055F89F5AB8086081F672AED5
:105CA0003092C928C4CD3E54A76577839FB3AF9582
:105CB0007745405B15F9121655C3E0A6BBF54AF1CE
:105CC000CC68F26347D08932A3ED1DBA60BE29DCEF
:105CD0009BA1F0DA17DAB049FD2DEB7F293A9D3709
:105CE00046D2901C2A8FDBD33E709AA84AD8E20E87
:105CF0002611142234512EDB2A5D65F8DA5881A86A
:105D0000CB1C3CB61A13FE9D0F3EEC6F30CA66A743
:105D10007714591D0717C02C46096E4825BE99D522
:105D200081651BD0A8E34EB84FB20FB761D50612FC
:105D3000A9ABFAAFC7FA27970FF9ADCE450E05917B
:105D4000A20BCF6A5B73C52235D65138EBDFC0B1E9
:105D50002F4F4B212EF35FB29878C0DA0BED37A4AA
:105D600056AFBF8D37FB7A9E7F820A90005E285B1C
:105D7000BD2529A6C575EA298A4712CDB439EA2579
:105D8000682E0ED80A5E87C66B6B3496155B26426A
:105D900011E856052729362936866101B8B8A1D5FC
:105DA0002496D70FE6C882C44BA214812A41637D92
:105DB00067339D8E3B2195BF48726B892ACD79AAA6
:105DC0003ED0EAB5BAD3214415CA86EB9B5E256264
:105DD0000ADCAD00162CE4D082F920E56A28545B79
:105DE00041EB053C47FBD6740CA99D4087849B384A
:105DF00026748D636681F04EBEA306AC7B1DF34F07
:105E000018A69D00E970CABA48DB6802ABD0F4CC92
:105E1000AF174EDA9056E7C3E02A86011944DC1129
:105E200039AF2E5034F91A02BE13A68F1C253BE35E
:105E3000F8240CB7DF7B258601A95151BBAD82C880
:105E4000F13AFA70D63A400DB5026297AE975D35D9
:105E5000C65F1C31D269321DAEA7D5B13E4127CFF6
:105E6000D9AC3709CA26262EEF9F0B8CED44F5BE20
:105E7000992173437097B2FB9D863C5C1A2C49AC08
:105E80002F09AC8E7267F6579DD40B8CAFEBE847A9
:105E900022A4AC286BB14BE4EC3BFF72150D10084B
:105EA0002FDD587705F18EC97050D6F76E2ADAA02B
:105EB000EEA911BA98482E653992664CB45896CF1F
:105EC000FAF86C3974E6DE18195B64EF3E484BDC77
:105ED000F74894211C9B76BE1DBC334A3561E9C549
:105EE000ACF57D60FCA80BF06359A41FAF3EB35026
:105EF000AADF89D74E5104F6276AC71F9DD57ED4E5
:105F0000257EF3B21FF81C2A3AA9FA34354E4417FD
:105F10002685061A268E2B29A30BE900727C5F7852
:105F200034D0F161B6D4E8ADC250A0003A53D9E5FF
:105F3000A0CD56884971EE7FD9BB7CE7CEB3CB119B
:105F4000872F93040AE255042DC930ABB9096A556D
:105F5000C98D567F646C583B5C455A902AFDF1957B
:105F60003C4763AF5068AECCD20B24A39B0E9B661C
:105F70000E311274809FF76675D7394414EB5CB606
:105F8000D7652E5C823C550A838675C5D97673F732
:105F90008F299A5578FBE1C6DAFA86C1E1BCC4C9FB
:105FA0001D9A2F967EBC703C8EE395EE02D9072396
:105FB000331C9E849A567D06F21E587336B8F38CB5
:105FC0001E29258D31D67B4569C4B2698FAC655ACF
:105FD0004F680C5CB231ED8731DE562F494F9F0F71
:105FE0007C16ADF11F26DCE81D68D475C947620137
:105FF0007E88A3E7F6971AEDAA0F8D9949AAEE8538
:10600000219B5DA20B2E1C32E79F3ADC253AD6CFAE
:106010002FC34EFF834E0AD2C967F3672E2CCF835E
:10602000FD0F171257DC8E75D0B9AE34A3C50382AD
:10603000EFE747773E10FBF4614FB0B9EB7726D41A
:10604000579CE5350868D8F9F46B0C86D9091DA86A
:106050001BCFC52ED99B543ED63626C9566DEEAA07
:10606000B3004C760E58130BDBB7B1D9DEB78C00FA
:1060700077F8284C45659B76E06EC3191EC1C3CBEB
:10608000D023D0FFA5A1E7820793B9458C094E4DD7
:10609000FBFF655BC80E376B1BA380043D43BA7DD5
:1060A00044910CA7585951B06B491A290E1580D745
:1060B0001C7518FD317AFF5E33D4748E1493050A73
:1060C000433F3260BDC108761E34B2812EB1D90D76
:1060D000680D93710CCC0A46BA1BCC88671D082F3B
:1060E000B9E315F1DC664C9B56F42F4868BCB2CE80
:1060F000964BC827396265366D2D21C3F05A4C6D19
:106100001EFA096440FCC0B44402D6D766FD5DE0C7
:1061100056845BAC61DAE24615D4B78657CA2903C8
:106120002F3460391E010F3390AA0EFDAD557892C1
:10613000D1D6B8DEF76EC86A2129B9CF89C0A8B513
:10614000CB473862B1FF010D5529AE004EC6BE6582
:10615000DB0D2CD2A543E6AB6D3E1416788A723364
:106160005D7F64F5FCF75F4154D8A8E694FEB69FC6
:10617000D5272D6B0304050A08060BFF0209070D3E
:10618000010C00FF202020205F5F7C002C006100BC
:1061900044697370206F66660D0A005553455200BE
:1061A00046004700424547494E0052414400442EB4
:1061B0004D590043005052474D0055534552202041
:1061C00020006620200067202000424547494E20DD
:1061D000202020200052414420202000442E4D59F0
:1061E0002020200043202020000D0C205A4B3B0093
:1061F000000D0C205A463F00000500000003072058
:1062000061853A0000FFFFFFFF4D000000C442001F
:10621000000000000051100000DC420000E14200DC
:1062200000DF420000FF00000029080000EB4200F0
:1062300000F5420000934200000000000049060003
:106240000007430000E1420000134300000000008B
:1062500000E906000015430000E142000021430070
:1062600000000000008108000023430000E142001C
:1062700000444300000000000011060000464300F7
:1062800000E14200000F000000F4010000040103DF
:10629000010201010411040F041704160118010082
:1062A00000BA610000C2610000C6610000CA61005E
:1062B00000A2610000D5610000DC610000E4610023
:1062C00000B5610000081C242C4448586C74050279
:1062D000050804080B08040405010504090809045D
:1062E0000608070206020402060106040701030865
:1062F00003040C080D020C0203020C010C040D0136
:106300000D080D0408020808070802020704080126
:106310000804090209010A080B020A0201080A011D
:106320000A040B01020802041008110210021108ED
:1063300010011004110112021201130213081208B5
:106340000F08120413011304140214011502150896
:106350001408170814041501150417021701190869
:106360001A0219021602190119041A011608160454
:106370001B021B081A0818021A041B011B04180828
:1063800018040B04202020202020202020200000A2
:1063900000010000009B610000A0610000A26100FC
:1063A00000A4610000A2610000AA610000AE6100CB
:0963B00000B3610000B5610000BA
:00000001FF
